:040000006F00905DA0
:10000400000000000000000090000020F60800201E
:10001400A9BDF9F5900000200000000000000000D8
:10002400900000209000002000000000000000006C
:1000340004120000000000009000002000000000F6
:10004400DC01002090000020B60100209000002078
:10005400900000209000002090000020000000008C
:1000640090000020900000209000002092000020CA
:10007400F201002090000020900000209000002059
:1000840090000020900000209000002090000020AC
:1000940001A01971175500E01305450DA2DE974024
:1000A40000E0E78000ED37340040834544401755B5
:1000B40000E01305250CBD89974000E0E780C0D916
:1000C400834744401147BD8B638DE7066369F7009E
:1000D4000947638DE70C7654096173002030194792
:1000E4006388E7043147E398E7FE175500E01305FA
:1000F400650A974000E0E780C0E783C7818317352E
:100104000000130565E13E95973000E0E780400666
:1001140083C58183AA9593F5F50F6800238CB1827A
:10012400973000E0E78040028547A38CF18265B7F1
:10013400175500E01305C504974000E0E78060E32D
:1001440059BF175500E013056504974000E0E780A8
:1001540040E21947A3050100B73600408347B100C8
:100164006316F7020346B10003C481831735000008
:10017400130585DA22956C00974000E0E78060C2A1
:100184008347B1003E94238C8182B1B78347B10089
:1001940003C686408C18AE97238EC7F88347B100F8
:1001A400850793F7F70FA305F1004DBF175500E03E
:1001B400130505FF51B7175500E0130565FF974078
:1001C40000E0E78000DBB71700400967239FE708DA
:1001D400973000E0E780C083730020303727004069
:1001E40083476700858B81C785472303F700730026
:1001F40020300145973000E0E78080AF85471755F0
:1002040000E01305A5FC238CF180974000E0E78013
:1002140040D6730020304111814601468145114585
:1002240006C6EF007004B727004011472383E78018
:10023400B7F700E003A707D16D9B23A8E7D003A776
:1002440007D15D9B23A8E7D0730050100100010083
:10025400B240410182800111814601468145114528
:1002640006CEEF007000B727004011472383E780D4
:10027400B717004083C6E70203C5E70413078008E5
:1002840093F6C60F1365350093E6160073360780A0
:100294001376860832C0010001009305700523809F
:1002A400B704130680FA2380C704010001002382E7
:1002B4000702238007040248732808800100010014
:1002C400733807801378880842C201000100238034
:1002D400B7042380C704010001002387D7022387C2
:1002E400A704238007049246F3A6068001000100B8
:1002F400F336078093F6860836C401000100238094
:10030400B7042380C7040100010083C6B70493E641
:100314000602A385D70423800704A246F3A6068019
:1003240001000100B7F600E003A506D113654500FE
:1003340023A8A6D003A506D15D9923A8A6D073004F
:1003440050100100010073370780137787083AC6FD
:10035400010001002380B7042380C70401000100C9
:1003640003C7B7041377F70DA385E70423800704B5
:10037400B247F3A7078001000100F24005618280C3
:100384003971B7F5070022DC81462A843010E10573
:10039400194506DE02D423160102F925B7170040D9
:1003A40083C6E70203C5E7041307800893F6C60F64
:1003B4001365350093E616007336078013768608B6
:1003C40032C601000100930570052380B7041306AB
:1003D40080FA2380C70401000100238207022380DE
:1003E400070432487328088001000100733807802D
:1003F4001378880842C8010001002380B7042380D1
:10040400C704010001002387D7022387A7042380A0
:100414000704C246F3A6068001000100F3360780F4
:1004240093F6860836CA010001002380B7042380AE
:10043400C7040100010003D50702F176FD16E98E19
:100444002390D70223800704D246F3A60680010036
:10045400010037F500E0832605D193E64600232802
:10046400D5D083D607026575110593F60660C18E53
:10047400C98EC206C18273350780137585082ACCDC
:10048400010001002380B7042380C7040100010098
:1004940003C5F70013650504A387A7002390D702BB
:1004A40023800704E246F3A606800100010091665A
:1004B400758C1DE873370780137787083ACE0100DF
:1004C40001002380B7042380C7040100010003C78F
:1004D400B70413670702A385E70423800704F247E0
:1004E400F3A707800100010037F700E0832707D155
:1004F400DD9B2328F7D0730050100100010013077F
:100504008008F337078093F787083ED00100010085
:10051400B7170040930570052380B704130680FACB
:100524002380C7040100010003D50702F176FD16FC
:10053400E98E2390D702238007048256F3A606800F
:10054400010001000DEC73370780137787083AD256
:10055400010001002380B7042380C70401000100C7
:1005640003C7B7041377F70DA385E70423800704B3
:100574009257F3A70780010001005145ED2EF25078
:10058400625421618280397152D481462A8A01469B
:100594008145114522DC26DA06DE4AD84ED63714C8
:1005A4000040D9218347E4020347E404930480080C
:1005B40093F7C70F1367370093E71700F3B6048068
:1005C40093F6860836C601000100930970052300DE
:1005D4003405130980FA23002405010001002302D5
:1005E400040223000404B246F3A6068001000100BD
:1005F400F3B6048093F6860836C801000100230090
:10060400340523002405010001002307F402230715
:10061400E40423000404C247F3A707800100010097
:1006240013055002E128B7F700E003A707D11367C9
:10063400470023A8E7D073B70480137787083ACA22
:1006440001000100230034052300240501000100FA
:100654000347F40013670704A307E400230004041A
:100664005247732707800100010073B70480137792
:1006740087083ACC01000100230034052300240537
:10068400010001002167336AEA00231044032300B8
:1006940004046247732707800100010003A707D100
:1006A4005D9B23A8E7D07300501001000100814630
:1006B4000146814511454D2EF3B4048093F484081A
:1006C40026CE010001002300340523002405010087
:1006D40001008347640493E717002303F404230011
:1006E4000404F247F3A7078001000100F2506254AA
:1006F400D2544259B259225A2161828001111307FE
:100704008008F337078093F787083EC20100010091
:10071400B7170040930570052380B704130680FAC9
:100724002380C7040100010083C6B70493F6F60DC5
:10073400A385D704238007049246F3A6068001000C
:10074400010093760502D5CEF336078093F686082A
:1007540036C4010001002380B7042380C7040100CC
:100764000100B70614007D89558D88C7010001007A
:100774000100010023800704A246F3A606800100BD
:10078400010073370780137787083AC60100010018
:100794002380B7042380C704010001000100010085
:1007A4003727004093061005A303D780238007044E
:1007B400B247F3A707800100010093078008F3B74D
:1007C400078093F787083ECE01000100B717004069
:1007D400130770052380E704130780FA2380E704D6
:1007E4000100010003C7B70413670708A385E704E2
:1007F40023800704F247F3A7078001000100056185
:10080400828093760504BDC6F336078093F6860886
:1008140036C8010001002380B7042380C704010007
:100824000100B7061400938606047D89558D88C798
:10083400010001000100010023800704C246F3A661
:1008440006800100010073370780137787083ACACE
:10085400010001002380B7042380C70401000100C4
:100864003727004093062005A303D780238007047D
:10087400D24781B773370780137787083ACC0100D2
:1008840001002380B7042380C704010001009847B6
:100894001367070C98C723800704E24719BF0111A7
:1008A400814601468145114506CE7D2A930780087D
:1008B400F3B7078093F787083EC601000100B71716
:1008C4000040130770052380E704130780FA238090
:1008D400E7040100010003C76704136717002383BB
:1008E400E70423800704B247F3A70780010001004F
:1008F400F2400561828041118146014681451145DE
:10090400A52213078008F337078093F787083EC4AE
:1009140001000100B7170040130670052380C704C7
:10092400930680FA2380D70401000100FD55239625
:10093400B70223800704A245F3A505800100010046
:1009440073370780137787083AC6010001002380B4
:10095400C7042380D7040100010003C76704136799
:1009640017002383E70423800704B247F3A7078013
:100974000100010001A0BD473305F50201007D150A
:1009840075FD8280411122C426C206C6AA84014490
:1009940063179400B24022449244410182800504CA
:1009A4001305803E4204C13F4180DDB72303048028
:1009B40015472303E48001002302A4808280830777
:1009C4006480E3CE07FE230304808280830764806F
:1009D400E3CE07FE03454480828083076480E3CE30
:1009E40007FE2302A4808280411126C44AC24EC05D
:1009F40006C61377F50BAD47AA892E89954463067D
:100A0400F70019456537653F8D444E854537FD59D7
:100A1400FD1463983401B240A24412498249410151
:100A24008280135509011375F50F453F2209CDB78F
:100A3400011126CC06CEB704080051371545BD3741
:100A4400713769372AC6A53F32459377150089EB7C
:100A5400136515001375F50FF240E24405618280B9
:100A6400FD14E9FC0145CDBF397126DC4ADA4ED8C4
:100A740052D656D45AD25ED006DE62CE66CCB7E7E2
:100A840000E07D5783AA070022C603AA470023A0DB
:100A9400E71823A2E718B71700401307700523804F
:100AA400E704130780FA2380E70483C74704930B02
:100AB40075FFB684E20793FBFB0F8546AA892E8B4C
:100AC400328937240040E187015763FA76016308CD
:100AD400D5008946130700026313D5000157D98F47
:100AE40093F7F70FB71C00402382FC04114723033C
:100AF400E4801305F00F5D3D094CD135636D7C1125
:100B0400B7050700DA9537870700795563F2E504DE
:100B1400B3879500636EF702370B0800A94733EBE0
:100B240065016399F90689E48144513D26850DA048
:100B3400DA850945553D05090345F9FFFD14050B03
:100B4400693D81C49377FB0FFDF7DD3569FD7D5564
:100B5400B7170040130770052380E704130780FAD2
:100B64002380E70403C74704418B2382E704F25040
:100B7400B7E700E023A0571123A24711E2543244FF
:100B84005259C259325AA25A125B825B724CE24CDD
:100B940021618280A5476395F90685691309F00FE1
:100BA400B3069900B3742B01B6941349F9FFB374D7
:100BB4009900856B33796901416B9387F9FFB3F72A
:100BC400270199E363FC340193D94900C147E3E663
:100BD40037FF99BF0569C1697D19D9B71305800D20
:100BE4006388690113050002638479011305100801
:100BF400CA85DD3B353D21DD4E99B3843441D9B7F7
:100C0400DA852D45D533CA94E30099F205097D3B75
:100C1400A30FA9FED5BF9387F9FF93F7F70F63617D
:100C2400FC0C83C71C0413073008631FF704370741
:100C34000800636BEB04B3079B00B706100063F571
:100C4400D704334BEB0089476393F9068980D54970
:100C5400E38C04ECDA850945413B11090327C9FFFC
:100C640091472320E48003076480E34E07FE2303B7
:100C74003481FD17EDFBFD14110B81C49377FB0F39
:100C8400E9FF7D3371F5E1B5B717004003C7570499
:100C9400B70708001377070219E3B78707007955E8
:100CA400E378FBEA33079B00E3FFE7F855B5854794
:100CB400E382F9F2DA852D45053B9389F4FFE38558
:100CC40004E6293393F7390091EB83260480032744
:100CD400090093074900E39AE6E43E89CE84F1BF14
:100CE400B5476396F9001305900BC93135BDB1477B
:100CF4001305B00AE38BF9FE99476391F904B7052C
:100D04000800B365BB002D45C53181448D4BA14915
:100D1400753963967401832704802320F9008504C0
:100D2400E39834FF8327048013172B0163550700CE
:100D34002312F900D5BB2322F900FDB39D47639923
:100D4400F90281451305B0044531BD44232009004F
:100D540023220900FD599D3993F77400CA9703C7EC
:100D64000700FD14398D2380A700E39634FF6DBB83
:100D7400A1476392F9046D398144630D0B008D47DB
:100D84009304C0036308FB009304000563048B0110
:100D9400930440041375C507E30895D81945393100
:100DA40039390545213126850D3909453D3149310A
:100DB400E31C05D669BB91476399F90013056006E6
:100DC400F536F53E130590090DB7E38F09D4F154B8
:040DD400A9BB0000B7
:100DD800971100209381018817610020130101A257
:100DE8001305400097F5FF1F93854521170600203E
:100DF800130606FE63FAC5008322050023A05500EA
:100E080011059105E3EAC5FE175500001305859104
:100E1800970500209385C5FB1386418163FAC500B9
:100E28008322050023A0550011059105E3EAC5FEBC
:100E380013854181972500209385C51D6377B500EB
:100E4800232005001105E36DB5FEFD42739002BC39
:100E58008D4273904280930280087390023097F21B
:100E6800FF1F9382A21993E23200739052309702C7
:100E780000009382822673901234730020303D4321
:100E88002A876373C3029377F700BDEFADE59376C6
:100E980006FF3D8ABA960CC34CC30CC74CC7410722
:100EA800E36BD7FE11E28280B306C3408A0697023D
:100EB800000096966780A6002307B700A306B70030
:100EC8002306B700A305B7002305B700A304B7009E
:100ED8002304B700A303B7002303B700A302B70096
:100EE8002302B700A301B7002301B700A300B7008E
:100EF8002300B700828093F5F50F93968500D58D72
:100F080093960501D58D61B7939627009702000047
:100F180096968682E78086FA9680C1171D8F3E9640
:100F2800E374C3F8A5B7854723AAF18017450000E5
:100F38001305051C23AE01806F20507123AE01807C
:100F48008D4723AAF180174500001305A51B6F20C4
:100F5800F06F371700408327870A411106C693E7C9
:100F680007202324F70A854513050010EF10905930
:100F78008D4513050020EF10F058EF20C0140D45E3
:100F8800EF2080179D47954505452380F182EF2086
:100F98004018B240B7E700E03707000823A0E71081
:100FA800410182805D71A2C41744000013048422A9
:100FB8001C4086C6A6C217050020130565E1829766
:100FC8005C5801459304000C8297170600200346DD
:100FD80066E88145138581845D35294785473AD080
:100FE8001D473AD23EC623AEF184B147238EF1861F
:100FF80023A00188D1472382F1889307000223A404
:10100800F1889307000423A6F188938701819C4304
:101018002C0005453EC426CEEF00307A0145EF107E
:10102800A001174500001305A512EF20D0731C5C22
:1010380001458297F24713070008638AE70863654A
:10104800F70213070006638AE700130700076380A7
:10105800E708130700056393E7021C4CF94505658B
:1010680013055592829719A81307000A638DE704A0
:101078006365F704130700096387E7045C5C32457E
:1010880082973C40680082977C401385C18582978F
:101098003C443745B3931305057882977C448145D2
:1010A800014582973C48814535458297EF10C03D00
:1010B800B64026449644616182801307000B63841E
:1010C800E700E39D97FA1C4C9305200349BF1C4C8D
:1010D8009305700369B779711305800406D622D485
:1010E80026D24AD04ECE97F0FF1FE780E0609535B4
:1010F800AD220145EF10D01BB1466D469945814799
:1011080001471305807EEF10F020B7E700E03707AE
:10111800001023A0E71005450564EF10105C974404
:1011280000009384240BBD3D894923AA0180130440
:1011380084BB174900001309690283C7818191E3C1
:1011480001A0238C0180FC489705002083D5A5D0F9
:101158002E8581460146829723168100FC50B246AF
:10116800094695454A854EC48297C1BF97470000F6
:1011780093874706FC5F411106C639458297552873
:10118800494597F0FF1FE780601F0545EF1090085D
:10119800E920E9227D3BB240410129B5411191473F
:1011A80017450000130585F806C623AAF18023AE6B
:1011B8000180EF20505BB24041014DBF411195477E
:1011C80006C623AAF18023AE01804D37B2401745E9
:1011D80000001305E5F641016F20504723AE01805A
:1011E80041118947174500001305C5F206C623AA11
:1011F800F180EF20B045B24041018DBF1387C18116
:101208001C4385071CC38280B747004003C70700FB
:101218001377F70E2380E7002382A70037470040A3
:101228008347670093F70704E5DF0345470082809B
:10123800E1BF411185457D5506C6EF10B02C8545A7
:101248007D55EF10903689450965EF10B02BB240F7
:101258008945096541016F105035411122C4371481
:1012680000400327840C26C2856406C6458F2324C4
:10127800E40C8D450565EF10503389451165EF1075
:10128800D0320327840C896789455D8F2324E40CB9
:101298000965EF1090318D450965EF10703BB7E790
:1012A80000E03707040023A0E7108327840A8D4550
:1012B8001D65C58F2324F40AEF10D0242244B240C0
:1012C800924441016F109053B717004003A7470C91
:1012D800014583A7470A82804111514506C622C4A9
:1012E80026C23714004097F0FF1FE7806069032784
:1012F800C40C856413052003458F2326E40C97F05E
:10130800FF1FE780E0678327840CB2405145C58FF3
:101318002324F40C22449244410117F3FF1F670071
:101328002366411122C426C206C6371400409744DA
:101338000000938424FC9307A03E0327440C9316D3
:10134800170163C70600B2402244924441018280DB
:10135800FD17E5F72685EF201041F1BF411106C6BC
:1013680022C426C24AC09307000873900780010070
:1013780001009307000C97140020938464B923900C
:10138800F40037140040713F0327C40A0569336726
:1013980027012326E40A03C50400593D03C51400A8
:1013A800413D8327840AB3E727012324F40A953FA4
:1013B800930780087390078001000100B24022441F
:1013C800924402494101828001119717002023812C
:1013D800A7B44AC82A8917150020130575B306CE85
:1013E80022CC26CA4EC693041600EF20D01A153F09
:1013F800371700408327C70A8566C204D58FC18086
:101408002326F70A014497190020938969B0636578
:101418009402371700408327870A8566D58F2324CF
:10142800F70A930740086302F9026244F240D24483
:101438004249B2490561F5B5B387890003C507007C
:1014480005041374F40FED33D9B7F2406244D24463
:101458004249B24905618280797126D293042600F7
:10146800C204971700202385A7AA97170020A381F5
:1014780007AA171700201307A7A94AD04ECE06D6E9
:1014880022D452CC2E89C1808147BA890507639B33
:10149800C70432C67935371700408327C70A8566DF
:1014A8000144D58F2326F70A170A0020130A4AA6F3
:1014B8003246636F94024A8597050020938565A597
:1014C800EF20700D371700408327870A225485665E
:1014D800B25092540259F249624AD58F2324F70A2E
:1014E800456181B58507C207A3000700C18379BF9D
:1014F800B387890003C5070032C61D3BB3078A00BE
:1015080005042380A7001374F40F5DB7E14717178C
:101518000020230FF79E93578500411117170020CD
:10152800A308F79E971700202385A79E171500206C
:101538001305359E06C622C426C24AC09304360047
:10154800EF207005F93B371700408327C70A8566E7
:10155800C204D58FC1802326F70A01441719002039
:101568001309099B63609402371700408327870A91
:1015780022448566B24092440249D58F2324F70A53
:10158800410145B3B307890003C507000504137477
:10159800F40F7939C1BF0111A307B10005469305BE
:1015A800F10006CEA537F24005618280E5477971E2
:1015B80017170020230EF79493578500171700205C
:1015C800A308F79426D293044600C2049717002074
:1015D8002381A79497170020A38D0792171700203F
:1015E800130707934AD04ECE06D622D452CC2E8962
:1015F800C1808147BA8905076398C7043717004037
:101608008327C70A85660144D58F2326F70A170A58
:101618000020130AEA8F634F94024A859705002039
:101628009385458FEF202077371700408327870A57
:1016380022548566B25092540259F249624AD58FB3
:101648002324F70A4561F1B98507C207A3010700FA
:10165800C18355B7B387890003C5070032C6C93EA1
:10166800B3078A00050462042380A7006184324618
:101678005DB701119305F100054606CE053FF2401E
:101688000345F100056182804111E94717150020E3
:101698001305258817170020231CF78606C622C4C1
:1016A80026C24AC093042600EF20E06E9D39371702
:1016B80000408327C70A85660144D58F2326F70A89
:1016C800171900201309C984634094023717004092
:1016D8008327870A22448566B24092440249D58FFF
:1016E8002324F70A410135B9B307890003C5070068
:1016F80005046204353E6184C1BFED471717002019
:101708002308F780931606017971C1829717002084
:10171800A380A78097070020238D077E1707002046
:101728001307077F26D24AD04ECE06D622D452CCF3
:10173800AE84138936008147BA89050763E9D7065D
:1017480032C6C536371700408327C70A8566324632
:10175800D58F2326F70A014417FAFF1F130A4A7B7D
:10176800B387890003C5070032C6D934B3078A0096
:1017780005042380A7001374F40F3246E36224FFA4
:10178800268597F5FF1F9385D578EF20C06037171A
:1017980000408327870A22548566B2509254025922
:1017A800F249624AD58F2324F70A45619DBE850711
:1017B800C20723010700C18349B739BE23AAA18202
:1017C80013854180DDBF81450145F1B34111130502
:1017D800301506C622C4713D2A8413054015513DB3
:1017E80093178400B24022445D8D42054181410136
:1017F800828001119305F1001305000C054606CE01
:10180800A30701009139F2400345F1000561828088
:101818009387818288438280937715001375F50F2B
:1018280013171500118B8E07D98F13573500058BA9
:101838000581D98F098901115D8DA307A100930541
:10184800F10005461305400806CE23A40182AD3EEB
:10185800F2400561828001112AC66C000546130515
:10186800000806CE9536B247F240B337F000850738
:1018780023A4F18205618280411101468145130547
:10188800100C06C69136B2408D4723A4F18241015F
:101898008280011193D785002304A100A304F100DD
:1018A8002305B100935786002306C1002C00154676
:1018B8001305400906CEA305F1003936F2409547D5
:1018C80023A4F182056182804111014681451305F7
:1018D800500C06C6D53CB240994723A4F182410179
:1018E8008280014681451305100DF9BC01468145EA
:1018F8001305200DD1BC01112AC623A6A1826C00B4
:1019080005461305A00806CEC134F2400561828061
:101918009387C18288438280011106CEEF20E03987
:1019280097470000938707BA9043D443EF103006D7
:10193800EF20E02B935705012306F1002307A100B0
:10194800935785006C000D4613056008A306F10047
:10195800A53CF24005618280011149052306A100DA
:10196800A306B10009466C001305E00806CEA93CA1
:10197800F2400561828001112AC66C0005461305F4
:10198800800806CE9134F240994723A4F18205617C
:10199800828001112306A100A306B10009466C004C
:1019A8001305F00806CE0D34F2400561828001115E
:1019B8009387C18222CC9C432A84084106CE6303C4
:1019C800F500153F1C403D476360F70417470000CA
:1019D8001307C7938A07BA979C43BA9782875C40D4
:1019E8002306F1001C44A306F1005C442307F10020
:1019F80021A81C48184C2306F1005C482307E10085
:101A0800A306F10023A2F1826C000D461305B0086D
:101A1800EFF09F9BF2406244056182805C4C230694
:101A2800F1001C50A306F1005C50C9B71C542306F2
:101A3800F1005C54A306F1001C584DBF23160100A9
:101A480023070100D1B701119387C18222CC9C439F
:101A58002A84084106CE6303F500713D1C403D47CA
:101A68006361F704174700001307478E8A07BA9780
:101A78009C43BA9782875C402304F1001C44A3046A
:101A8800F1005C442305F1001C48A305F1008347DD
:101A980044012306F1001C4CA306F1005C4C23070B
:101AA800F1002C001D461305C008EFF0FF91F2402D
:101AB80062440561828083470402A306010023046F
:101AC800F1005C50A304F100834784022305F10070
:101AD8005C54A305F1001C582306F10023070100FC
:101AE800C9B75C582304F1001C5CA304F1005C5CDA
:101AF8002305F1003C40A305F10083474404230675
:101B0800F1003C44A306F1007C4451BF3C48230447
:101B1800F1007C48A304F1003C4C2305F1007C4C07
:101B2800A305F1002316010055BF02C4E5BF797172
:101B380022D452CC2A842E8A09466C005D4526D2CE
:101B48004ECE06D64AD0EFF03F919387C18283A943
:101B580007000547BE846394E904056913053990B5
:101B6800093E1D811375F50F631B35031305199085
:101B780009362300A4008345040017450000130517
:101B88006589EF20A02C8347D100B250225423004E
:101B9800FA0092540259F249624A4561828094409F
:101BA80011478347C1006393E60089072300F400C7
:101BB800D9B7011122CC15462A842C00754506CECA
:101BC800EFF09F899387C1829C433D471CC06360A7
:101BD800F70C173700001307677B8A07BA979C43EF
:101BE800BA97828703478100834791008946334724
:101BF800D702B3C7D7023307E0402302E400B30794
:101C0800F0400347A100A302F4009357670013F6BE
:101C180017008347640093564700898A93F7C70FD4
:101C2800D18FD58F93562700918A93F7370F137664
:101C38008700D58FD18F1316270093164700418A46
:101C480093F7F70C93F60602D18FD58F058B1A07F9
:101C580093F7F7FBD98F0347B1002303F400935799
:101C6800570093F6170083477400058B060793F710
:101C7800C70FD58FD98FA303F4008347C10013F78B
:101C8800770083478400E19BD98F2304F400F24056
:101C9800624405618280834781000947B3C7E70230
:101CA800B307F0402302F40083479100139787019C
:101CB8006187634407008983A9B7938707F01147B1
:101CC800B3C7E702E207E1872DBF034781008946D2
:101CD800834791003347D702B3C7D7023307E040A1
:101CE8002302E4000347A10093564700898AB307FB
:101CF800F040A302F4009357670013F617008347D8
:101D0800640093F7C70FD18FD58F93562700918A18
:101D180093F7370F13768700D58FD18F13162700C7
:101D2800418A9316470093F7F70C93F60602D18F72
:101D3800D58F058B1A0793F7F7FBD98F2303F40088
:101D48000347B10083477400135667009356370062
:101D580093F7870F918AD18FD58F93561700058BEC
:101D6800A18A93F7770E120729B70347810089469E
:101D7800834791003347D702B3C7D7023307E04000
:101D88002302E4000347A10093564700898AB3075A
:101D9800F040A302F4009357670013F61700834737
:101DA800640093F7C70FD18FD58F93562700918A78
:101DB80093F7370F13768700D58FD18F1316270027
:101DC80093164700418A93F7F70C93F60602D18FD2
:101DD800D58F058B1A0793F7F7FBD98F2303F400E8
:101DE8008347B10013F7170083477400F99B59B56F
:101DF8002146814513054400EFF06F88BD471CC09C
:101E080079B501119305F1007D45054606CEA30776
:101E18000100EFF06FE40345F1008947F2403345D4
:101E2800F50205613305A04062056185828093173C
:101E3800850021815D8D93978500A181DD8D9317A4
:101E48008600218201115D8E93978600A18223145A
:101E5800A1002315B1002316C100DD8E2C002146F8
:101E68001305D00806CE2317D100EFF0EFD5F240C6
:101E78000561828001116C005545094606CEEFF0D8
:101E8800AFDD8347C1000345D100F240A2075D8D55
:101E98000561828093178500218101115D8D2316CC
:101EA800A1006C0009461305700906CEEFF0CFD1EA
:101EB800F2400561828001111375F503A307A100A3
:101EC8009305F10005461305900806CEEFF0CFCF35
:101ED800F2400561828001112AC66C00054613058F
:101EE800600906CEEFF04FCEF240056182800146D0
:101EF80081451305500D6FF02FCD1305F5FD931790
:101F0800850042054181218101115D8D2316A100C3
:101F18006C0009461305800906CEEFF0EFCAF240BF
:101F28000561828001116C0009461305800906CEFF
:101F380023160100EFF04FC9F240056182800111BC
:101F4800A307A1009305F10005461305E00906CE95
:101F5800EFF08FC7F240056182800111A307A1004D
:101F68009305F10005461305B00906CEEFF0CFC57D
:101F7800F240056182802E86AA8501456FF0CFF078
:101F8800797122D42E8426D29305F101AA84228560
:101F980032C606D6693E8347040032460545636962
:101FA800F6000345F1013E86A685EFF00FF50145E1
:101FB800B25022549254456182801387C1821843DB
:101FC8008D46AA87630ED7029146630DD70405454F
:101FD8003DE3FD1793F7F70F0947636EF70486078C
:101FE800173700001307C772BA9703D507001546BD
:101FF800411106C6EFF08FD1B24001454101828000
:102008009307F5FF93F7F70F094705456365F7024F
:1020180086071737000013072770BA9703D50700FC
:102028001146F9B7054705456397E7000565114669
:102038001305F59C75BF8280411126C2856422C4B0
:102048002A841385D49C06C6EFF0AFE23D889375C9
:10205800050FC18D2244B2401385D49C924441019E
:102068006FF06FD39317850021815D8D9387C182AF
:102078009C43011106CE2316A10081C70D47639921
:10208800E700056509466C001305859CEFF00FC84D
:10209800F24005618280411122C4056426C293552D
:1020A8008501AA841305F49C06C6EFF0CFCE93D51C
:1020B80004011305049D93F5F50FEFF0CFCD93D5EB
:1020C80084001305149D93F5F50FEFF0CFCC13059D
:1020D800249D2244B24093F5F40F924441016FF0DD
:1020E8008FCB37C5898E130565ED75B793178500B6
:1020F80021815D8D9387C1829C43011106CE2316F1
:10210800A10081C70D476399E700056509466C0082
:102118001305659CEFF08FBFF240056182809387BD
:10212800C18298439147AA8563ECE7008547B39736
:10213800E700E58B91C705651305559C6FF0AFC5A2
:102148008280411122C405641305F48906C6EFF0A4
:102158004FD2936505F893F5F50F1305F489EFF061
:102168008FC313055489EFF0CFD09375E50F13058E
:1021780054892244B24041016FF0EFC1411122C499
:1021880005641305F48906C6EFF0AFCE9375F5071D
:102198001305F489EFF02FC013055489EFF06FCDC4
:1021A80093651500130554892244B24093F5F50F41
:1021B80041016FF04FBE411122C4056426C2AA84B2
:1021C8001305E48906C6EFF0CFCA9375050F13050A
:1021D800E4892244B240C58D924441016FF0AFBBFF
:1021E800411106C622C405C58547631AF502056470
:1021F80013051489EFF0EFC7936505FC93F5F50F08
:10220800130514892244B24041016FF0CFB8056428
:1022180013051489EFF0EFC59375F503D5B7B240F0
:102228002244410182809387C18298438947631F72
:10223800F702411126C2856422C42A8413851493A7
:1022480006C6EFF00FC3916793156400938707FCE8
:102258001375F5032244FD8DC98DB240138514937F
:10226800924493F5F50F41016FF0EFB282800111AE
:10227800935785012306F10093570501A306F10042
:10228800931785004205418121815D8D9387C18225
:10229800984306CE2317A10089476319F7000565FF
:1022A80011466C0013056591EFF04FA6F2400561E9
:1022B80082800111935785012306F1009357050188
:1022C800A306F100931785004205418121815D8DA8
:1022D8009387C182984306CE2317A10089476319C3
:1022E800F700056511466C0013052591EFF00FA264
:1022F800F240056182804111054506C622C4056485
:10230800EFF06FD51305F497EFF0AFB6936525009E
:1023180093F5F50F1305F497EFF0EFA71305449223
:10232800EFF02FB59375F50C13054492EFF0AFA6B7
:10233800130544962244B24041016FF08FB393874E
:10234800C182984389476318F702411126C2856400
:1023580022C4935585002A841385C49206C6EFF0DB
:102368008FA39375F40F2244B2401385D4929244FC
:1023780041016FF04FA28280411122C40564130508
:10238800349206C626C2EFF0CFAE93650502AA8442
:1023980093F5F50F13053492EFF0EF9F1305349280
:1023A8002244B24093F5F40D924441016FF0AF9E80
:1023B8009307F0079375F50F6374F5009305F0071D
:1023C80005651305E5916FF00F9D01112306A10026
:1023D8006C0005461305300A06CEEFE0FFFEF2401A
:1023E800056182807971C205C181230EA100416512
:1023F80093D785007D15A30EF10006D6230FB100F3
:10240800EFF05FA99387C182984389476314F70067
:102418000545653F6C080D4613053008EFE0DFFA07
:10242800B250914723A4F18245618280011106CE02
:1024380032C436C689362245B245F24005615DB7D9
:102448007971C205C181230EA100416593D785002A
:102458007D15A30EF10006D6230FB100EFF09FA360
:102468009387C182984389476314F7000145B13FB8
:102478006C080D4613052008EFE01FF5B25095478C
:1024880023A4F1824561828085472388F182828076
:10249800938741829C4361476386E7026367F7003D
:1024A80029476386E7020145828013076002638536
:1024B800E70213074003E398E7FE372503001305F7
:1024C8005597828037650C001305455D828037D5A6
:1024D8001800130585BA8280373506001305A52E26
:1024E80082809387C18298438947631BF70E411105
:1024F8004AC02A89054506C622C426C28564EFF06B
:102508008FB51385F497EFF0CF969365250093F573
:10251800F50F1385F497EFF00F8813854492EFF0C9
:102528004F959317490093F707039375F50CDD8DC5
:1025380013854492EFF02F8613851496EFF06F936E
:102548002A8413852496EFF0CF9222054204498C01
:1025580013853496EFF0EF91498C0145EFF0AFAF5A
:10256800630B09028D470145814563E527072285ED
:10257800EF10A074973700009387C7E89043D443BF
:10258800EF10E01B97370000938747E89043D44348
:10259800EF00F03F81A0B70780006345F400B7075C
:1025A80000FF3E94F5352A892285EF10006A2A84B7
:1025B8004A85AE84EF1060692A86AE862285A68594
:1025C800EF00F03C97370000938747E39043D443EC
:1025D800EF10E016B2402244924402494101828041
:1025E8000145814582809387C1829C430547FD1739
:1025F8006364F70A41114AC005691305499506C67F
:1026080022C426C2EFF0EF862A8413055995EFF00D
:102618004F86AA84420413056995A204EFF06F85DA
:10262800458C418DB70710001384F7FF1317C500B9
:10263800698C635307001D8CA13D2A892285EF1000
:10264800C060973700009387E7D99043D443EF10D1
:10265800000F2A844A85AE84EF10205F9737000068
:102668009387C7D82A86AE868843CC43EF0030329A
:1026780097370000938707D89043D443EF10200C76
:102688002A86AE862285A685EF007030B2402244A5
:102698009244024941018280014581458280238814
:1026A80001828280411126C2938481829C4006C6A1
:1026B80022C44AC06382073483C701839DC383C78A
:1026C8001182638B0732930700087390078001001B
:1026D8000100A3800182930780087390078001009E
:1026E80001009387C18203A90700EFF0AFF82A849D
:1026F80041657D15EFF00FFA914763E02721173701
:1027080000001307A7CC0A093A9983270900BA974A
:1027180082879C401147638BE7081547639FE71C36
:10272800937724009374840099CB9387418313771C
:1027380004049C4325C381C79C4F0945ADE39377A7
:10274800440081CB938741839C4381C79C4791C3B5
:10275800829789C8938741839C4389C79C4F99C3B3
:10276800054582979317140163D90700938741831E
:102778009C4381C7DC4B91C382970588630F04167D
:10278800938741839C43638A07169C436387071694
:102798008297A5A299C4C5D79C4FD5D305458297E2
:1027A80079BFD1DFDC43C1DF829751BF9377140033
:1027B80081CB938741839C4381C79C4391C3829774
:1027C8009317140163DB0712938741839C43638645
:1027D80007129C4B65BF9C4015476389E70419475E
:1027E800638EE70E1147639AE7101735000013054B
:1027F80065C6EF1040779377140091CF1735000026
:10280800130545C7EF102076938741839C4381C702
:102818009C4391C382979317140163D0070E173511
:102828000000130565C7EF10007479BF1735000065
:10283800130585BFEF102073EFF0CFE3AA85173596
:102848000000130525BFEF1060609377240095C33F
:1028580017350000130505BFEF10E07093770404E7
:1028680013874183B5C71C4389C79C4F99C3094542
:1028780082979377040181CB938741839C4381C7D7
:10288800DC4791C382979377040289CB938741836E
:102898009C4389C79C4F99C301458297931714019C
:1028A80063D90700938741839C4381C7DC4B91C35D
:1028B800829793770410E38207EC938741839C43C4
:1028C800E38D07EA9C4FE38A07EA0D45829775B5C1
:1028D8001C43C5D3DC43D1DF829761BF9317340112
:1028E80063DE070293874183131724019C436351D6
:1028F800070281C79C53054585E32244B2409244B0
:102908000249173500001305A5BA41016F10A065EB
:10291800EDD79C53FDD301458297C5B79317140192
:10292800E3DD07FC938741839C43E1DBDC4BB9BDC6
:102938009C4011476389E7081547E390E7FC9377C4
:10294800041089CB938741839C4389C7DC4F99C383
:10295800014582979317440163DA070093874183FF
:102968009C4389C7DC4F99C3054582979377040830
:1029780089CB938741839C4389C7DC4F99C305451D
:1029880082979317140163DA0700938741839C4366
:1029980089C7DC4F99C3014582979377040181CB9E
:1029A800938741839C4381C7DC4791C38297137403
:1029B800040221D4938741839C43A1D39C4F0145B2
:1029C8008DDF82971DBF9377044089CB938741831E
:1029D8009C4389C7DC4F99C3094582971374042027
:1029E800E30D04F0938741839C43E38807F0DC4FB1
:1029F800E38507F00D45F1B7B240224492440249FD
:102A08004101828083C7018389C78547A380F182FA
:102A1800828049B9B717004003C7E7040D894111FF
:102A28001377C70F498F93068008F3B6068093F68D
:102A3800860836C601000100930670052380D70476
:102A4800930680FA2380D704010001002387E70456
:102A580023800704B247F3A7078001000100410162
:102A68008280B717004003C7E7020D894111137729
:102A7800C70F498F93068008F3B6068093F6860839
:102A880036C601000100930670052380D70493061B
:102A980080FA2380D704010001002387E7022380FE
:102AA8000704B247F3A707800100010041018280B3
:102AB800011122CC06CEB717004083C7F70293F75F
:102AC800F70F13E4470009E5054513F4B70F513F25
:102AD80093078008F3B7078093F787083EC601007D
:102AE8000100B7170040130770052380E704130798
:102AF80080FA2380E70401000100A387870223806E
:102B08000704B247F3A7078001000100F2406244BE
:102B18000561828041112A83014E930E407E130F76
:102B28000019930F400663E56E129308001913030A
:102B38004006B3781503854E0D4FA14F33736502D8
:102B48000D891335150063EFBE121308F6FF794699
:102B580072984208135808013307C70213D61700A2
:102B6800BE0732976146B3F6C60213068070B38675
:102B7800C6023697A166F58F42075D8FB7160040EB
:102B880083C7F60293F70708A303F1000346710011
:102B980083C7F60293F70708E394C7FE83477100DB
:102BA800B716004093F7F70F63880712930780085A
:102BB800F3B7078093F787083EC401000100B717F1
:102BC8000040930670052380D704930680FA23807B
:102BD800D7040100010023AA070383C6170393E65D
:102BE8000608A388D70223800704A247F3A7078013
:102BF800010001001166B71700407D16D45BC85F5D
:102C080093854703A98EF18EF5FA93068008F3B6EB
:102C1800068093F6860836C6010001009306700503
:102C28002380D704930680FA2380D704010001008B
:102C380098C103C7170313670704A388E702238013
:102C48000704B247F3A70780010001004101828011
:102C58007D133368E3039308E016630E08003368B6
:102C6800F3039308D016630808009378330093B8E9
:102C780018009388D81633081E01131E0801135E26
:102C88000E0155B56393E5030548638608000148BE
:102C9800630303002A8871087298FD15131E080142
:102CA800C205135E0E01C18179BD13F8150063F4E6
:102CB800BF007908D5B713381800E5BF83C7F602F7
:102CC80093F70708A303F1000346710083C7F602D0
:102CD80093F70708E394C7FE8347710093F7F70F4C
:102CE800F1DFE9B509C58547630AF5008280B717A2
:102CF8000040130700022388E7028280B7170040CC
:102D08004147D5BF914763EEB70217270000130765
:102D1800E77B8A05BA959C41BA978287B717004026
:102D280003A7470B1345F5FF698F23AAE70A03A7F3
:102D3800070B698F23A8E70A03A7070A798D23A041
:102D4800A70A8280B717004083A6470B1347F5FFF1
:102D5800F98E23AAD70A83A6070B558D23A8A70A9D
:102D680083A6070A758F23A0E70A8280B717004059
:102D780003A7470B498F23AAE70A03A7070B1345A5
:102D8800F5FF45BFB717004083A6470B1347F5FF6C
:102D9800758F23AAE70A03A7070A598D4DB7B717F6
:102DA800004003A7470B498FEDB7914763EEB70281
:102DB800172700001307C7728A05BA959C41BA976E
:102DC8008287B717004003A7470D1345F5FF698FA2
:102DD80023AAE70C03A7070D698F23A8E70C03A70D
:102DE800070C798D23A0A70C8280B717004083A613
:102DF800470D1347F5FFF98E23AAD70C83A6070DB5
:102E0800558D23A8A70C83A6070C758F23A0E70C64
:102E18008280B717004003A7470D498F23AAE70C04
:102E280003A7070D1345F5FF45BFB717004083A655
:102E3800470D1347F5FF758F23AAE70C03A7070C67
:102E4800598D4DB7B717004003A7470D498FEDB708
:102E58009357E50093F70730C98FC2070547C18329
:102E68006382E5048DC10947638DE5040D476380DE
:102E7800E50637170040231FF70883562709D58F23
:102E88002319F7088280371700400356670993C64D
:102E9800F7FFF18E231BD7088326C70C558D2326F1
:102EA800A70CC1BF371700400356670993C6F7FF41
:102EB800F18E231BD7088326870C558D2324A70C56
:102EC8004DBF3717004083566709DD8EE1B73717C6
:102ED800004083566709DD8EE9BF797122D4371423
:102EE800004026D24AD0035924028354040206D64D
:102EF8004209C2044ECE52CC56CA13590901C180A8
:102F08002DE11379F9F793F4F49F4209C204135998
:102F18000901C18093078008F3B7078093F78708F2
:102F28003EC401000100930770052300F4049307D1
:102F380080FA2300F4040100010023112403231064
:102F4800940223000404A247F3A7078001000100AC
:102F5800B250225492540259F249624AD24A456107
:102F68008280B7F5070081463000B105194597E022
:102F7800FF1FE78020AFA24713972701E34A07FC0A
:102F88001369090893E4044093098008F3B709809A
:102F980093F787083EC001000100930A70052300DB
:102FA8005405130A80FA2300440501000100231187
:102FB800240323109402230004048247F3A7078004
:102FC80001000100294597E0FF1FE780809AF3B9C7
:102FD800098093F989084EC20100010023005405B5
:102FE80023004405010001008357040293E70720EA
:102FF8002310F402230004049247B9B7B7470040EE
:103008001147A381E70009472380E700130700065B
:103018002380E70003C7170013670701A380E700B1
:1030280003C717001377E70FA380E7008280B7175D
:1030380000408847420541819377050491EB9377D7
:10304800F5013755E801130505803345F5028280FF
:103058009377050C130700046397E7009377F5014E
:1030680037459C1CCDB72165130505D08280814763
:1030780037370040A14663C4C700328582800345C4
:10308800B740E38EA6FE3385F500034505008507A6
:103098002304A740CDB7411122C406C62A84413F64
:1030A8002947B307E502B2408D83B3D7870222448C
:1030B8009507B3D7E70237370040C207C183231605
:1030C800F74041018280716541111305052006C64C
:1030D800D937B7370040130770F82381E7400D4709
:1030E800A381E74013070004A380E740054723872F
:1030F800E740B2404101828037370040834727408C
:103108001A0593F7F703C98F93F7F70F2301F740D1
:103118008280B737004003C7174019C9D98DA380EB
:10312800B74003C70740136787002380E7408280C2
:1031380093C5F5FFF98DA380B7408280B73700406B
:103148002147B736004091E1828003C6B740E30CBF
:10315800C7FE05050346F5FFFD15C2052384C640D5
:10316800C181D5B78147B736004003C7A64013963B
:10317800070141821377F70F19E33285828003C66E
:1031880086403307F50085072300C700F9BF39716A
:1031980093D7450122DC4AD856D22A891394C50010
:1031A80006DE26DA4ED652D45AD05ECE13F5F77F15
:1031B800318093DAF501630B05109307F07F630BF9
:1031C800F514135AD9010E0433648A00370A8000B3
:1031D800336A4401131B3900930415C00144814B21
:1031E80013D846011399C6001378F87FB28813598B
:1031F800C90093D9F601630E08089307F07F6300AE
:10320800F8041357D6010E0933692701130818C0AB
:10321800B70780003367F90093183600B384044178
:103228008145BD4733C83A0163E4871A97270000F0
:103238009387472C0A043E9410403E9602863367D3
:10324800C900938414806312071013642400814812
:103258008945C1BF1306F07F81470147B207F25085
:1032680062545206B1837E08D18FB3E70701D25466
:103278004259B259225A925A025BF24B3A85BE859C
:103288002161828001481306F07FB70708000147D3
:10329800F1B73367C9004DC7630709304A8532C49F
:1032A800EF0010282246130755FFF547930685FFC0
:1032B800998F3319D900B357F60033E72701B318AC
:1032C800D60026959304353F8145A1BF336A240172
:1032D80063030A0636C632C46306042A2285EF0051
:1032E80030242246B246AA84130755FF754A138B29
:1032F80084FF330AEA4033146401335A4901336ABC
:103308008A00331B69011305D0C0B30495400144FA
:10331800814BF9B5336A240163180A002144014B33
:103328009304F07F894B6DBD228A4A8B3144930404
:10333800F07F8D4B75B51144014B8144854B4DB5DC
:103348001364140081488545E9BD136434004A8735
:103358008D45C1BD6308052E8547898F9306800377
:1033680063DBF632014681470147CDBDCE868947EA
:10337800638BF53A8D47E387F5F085473688E38315
:10338800F5FE1385F43FE357A0FC93F778006394A8
:10339800072893D638009317770063D80700B70734
:1033A80000FFFD177D8F138504409307E07FE3C37B
:1033B800A7EA1316D70193179700B1833367D6008E
:1033C8001376F57F61BDD6865287DA88DE8545B7E4
:1033D800636F4721630BEA20DA86FD145284014BA0
:1033E8009317870013D388013363F300935E0301B7
:1033F800B357D403131F0301135F0F0193D50601BD
:10340800139E88003374D4033307FF024204C18D2E
:1034180063FBE5009A951386F7FF63EC652663FA6C
:10342800E526F9179A95998D33D7D503C206C18237
:10343800B3F5D5033306EF02C205D58D63FBC5008E
:103448009A959306F7FF63E4652463F2C524791718
:103458009A95C20741645D8F9307F4FF3375F700AF
:1034680093580701935F0E01B377FE00B302F5028C
:10347800B386C540B383F80293D502013386AF0201
:103488001E962E963385F803637376002295C168DD
:10349800FD1893550601337616014206B3F812015A
:1034A800AA95469663E4B6126380B6123306CB40FB
:1034B8008D8E333BCB00338B66411385F43F630A13
:1034C8006317B358DB0393550601337BDB03B3065D
:1034D8001F03420B33EB6501637BDB001A9B93856B
:1034E800F8FF636B6B206379DB20F9181A9B330BA9
:1034F800DB40B356DB0342064182337BDB03330FE9
:10350800DF02420B33666601637BE6011A969385F8
:10351800F6FF6365661E6373E61FF9161A96C208FE
:10352800B3E8D8009395080193D20801C181B38EFE
:10353800F5023306E641B385BF0293D60E01B38781
:10354800F202BE95AE96B38F5F0263F4F600C167D0
:10355800BE9FC165FD1593D70601ED8EC206B3FE69
:10356800BE00BE9FF696637DF6091A969387F8FF0C
:103578006367661A6366F619630DF61BBE8893E8DF
:10358800180011B54A85692F13075501F1459304B1
:1035980005022246B246E3DBE5D4130485FF331A5D
:1035A8008900014B8DB3328532C49D2F1307550115
:1035B800F146AA87224613050502E3D8E6CEE117AD
:1035C8003317F6008148F5B9E372CBEE729B3335B9
:1035D800CB011A95AA961305F7FF6378D30263E621
:1035E800B6106382D5102A87D1B5E3671BDF9355E0
:1035F8001B009316FA0113541A00CD8E7E0BCDB31F
:10360800E31FF6F7E38106D88DB7E31ED3FCE37812
:10361800CBFD2A8761BD93F7F8009146E38BD7D697
:1036280093B7C8FF9386480093C717008D823E97CB
:103638009DB381468547E34CA0FEFD58E31E05D0A7
:10364800930410C085471385E441B316A70033D609
:10365800F8003395A800D18E3335A000C98E13F633
:1036680076003357F70001CE93F7F60011466388CA
:10367800C70093874600B3B6D7003697BE86931720
:10368800870063D80704054681470147C1BE3687CE
:10369800C9B3B28749BBFD46E3D7F6FA0556098E8A
:1036A800930600023356C7006388D7009387E44324
:1036B800B317F700B3E8F800B3361001D18E13F64C
:1036C8007600814701CE93F7F60011460147E39251
:1036D800C7FA931797001316D701B18313D736008B
:1036E800518F0146A5BEE370CBF0729B3335CB01F9
:1036F8001A957917AA965DBBAE88D5BBAE8605B577
:1037080093171E0033BEC70172931A96F9183E8E9E
:10371800E317F6E7E309DEC693E81800ADB1BE8803
:10372800E30AF6FFA9BD36881306F07F81470147F3
:1037380035B6E367DEFCBE88E310DEFEA9B1397159
:103748004AD813D945014ED652D456D29399C500BA
:1037580006DE22DC26DA5AD05ECE1379F97F2A8A71
:1037680093D9C90093DAF501630D090E9307F07F29
:103778006304F9181354D5018E09B3693401370469
:10378800800033E4890093143500130919C0814976
:10379800814B13D74601139AC6001377F77FB2857A
:1037A800135ACA0013DBF601630A07109307F07F68
:1037B8006303F7049357D6010E0A33EA4701130748
:1037C80017C0B7078000B367FA00931536003A9917
:1037D800814833C76A01BD463A851308190063E674
:1037E8003617172600001306E6D48A09B29983A66D
:1037F8000900B2968286B367CA001309F97F6397F6
:10380800071293E9290081458948E1B701479307E1
:10381800F07F3704080081443204D20731807E07E4
:103828005D8C598CA285F250625426854259D25437
:10383800B259225A925A025BF24B216182805A8510
:103848003E84AE84C68B8947638BFB0E8D47E38F1E
:10385800FBFA85472A87639AFB38814701448144EC
:1038680065BF33E4A90055CC36C632C46389092A3A
:103878004E857D212246B246AA87130755FF754417
:10388800938487FF198CB399990033548A00336461
:103898003401B3149A0013D746011309D0C0139A00
:1038A800C6001377F77F3309F9408149814BB28508
:1038B800135ACA0013DBF601E31A07EEB367CA000E
:1038C800A9C7630E0A22528532C4992922462A873B
:1038D800930655FFF547930587FF958F331ABA006E
:1038E800B357F600B3E74701B315B6003309E9400B
:1038F8001309D9C08148F1BD33E4A90001ECA149FD
:1039080081441309F07F894B69B593E91900814512
:103918008548C1B54E84AA84B1491309F07F8D4BFF
:103928008DBD914981440149854BA5B593E939007D
:10393800D2878D4879BD89475685E399FBF02A8758
:103948009307F07F01448144C1BDC16E1386FEFF19
:1039580093D6040113DE0501F18CF18D33869502AF
:103968003383B6029358060133059E021A95AA9826
:10397800B382C60363F36800F692C16F1383FFFF37
:1039880033F5670093D30701B3F76800C2073373B1
:1039980066003E933306950293D80801B387A602C2
:1039A800135F0601B3849302BE94FA94B38E760231
:1039B80063F3F400FE9E416A9307FAFF935F0401E4
:1039C800B376F400B3F9F4007D8EC1803384D50258
:1039D800C209338FD401B299CE98B307DE02935E41
:1039E8000401B385BF02AE97BE9E330EFE0363F398
:1039F800BE00529EC1679385F7FF33F6BE006D8CFB
:103A08004206229693DE0E01B305D502769E3385D3
:103A1800AF0213D40501B386D302AA96A296B38F38
:103A2800F30363F3A600BE9F41657D15B3F7A600B7
:103A3800C2076D8DAA97B3855800B3B93501FA97B7
:103A4800B2953384370133B6C500B30EC40133854C
:103A5800CE0033343401B3B7E701C18F33BECE0192
:103A680013D406013336C5003E943366CE009394D2
:103A7800950032947E94B3E464002604935675014D
:103A8800B3349000DD8193179500CD8C558CDD8C77
:103A98009317740063DB070093D714008588931687
:103AA800F401DD8CD58C058042899307F93F635773
:103AB800F00893F6740081CE93F6F40011466388FB
:103AC800C60093864400B3B496002694B684931631
:103AD800740063D80600B70700FFFD177D8C9307B5
:103AE80009409306E07F63CDF60E93D63400931415
:103AF800D4012604D58C318093F7F77F31BB32850A
:103B080032C4392C93065501F147130705022246A2
:103B1800E3D2D7DC6115B317A6008145C1BB0924E0
:103B280013075501F145930705022246B246E3D82B
:103B3800E5D461153314AA008144B1BB85469D8E36
:103B4800B1E71309E941B3972401B3D4D400331979
:103B58002401B337F000B3649900DD8C93F7740047
:103B6800B356D40081CF93F7F40011466388C70099
:103B780093874400B3B49700A696BE8493978600B3
:103B880063D8070485470144814479B1130680034B
:103B9800E345D6CC7D46E356D6FA0556B307F6403C
:103BA800930500023356F4006387B6001309E9430E
:103BB800B3172401DD8CB3349000D18C93F67400D4
:103BC800014499CA93F7F40011468146E392C7FA73
:103BD800139496003180F6068D80D58C81472DB9D7
:103BE8009307F07F0144814405B942897DBD93D78D
:103BF8004501B70610001387F6FF93F7F77F130602
:103C0800E03F2A886D8F0145FD816354F60099C114
:103C1800828082801306E0417D55E34BF6FE130552
:103C280030431D8D7D46558F634AA6009387D7BEC6
:103C38003317F7003355A800598D8280130530419A
:103C4800B307F5403355F7008280411106C622C4F8
:103C580026C205CD9357F541B3C4A7009D8C2A848D
:103C680026857D289306E041898EA9477D8093F6B5
:103C7800F67F63CDA7022D47098FB3D7E40055051A
:103C8800B207B394A400B18329A0014481468147B7
:103C98008144B207D206B1837E04D58FC18FB2406A
:103CA80022442685BE859244410182805515B397EA
:103CB800A400B207B1838144E9BF15CD411122C4E4
:103CC80006C62A84B1289306E041898EA94793F64F
:103CD800F67F63DCA7025515B317A400B207B183BA
:103CE8000147B2402244B207D206B183D58F3A8544
:103CF800BE854101828081478146B207D206B183E1
:103D08000147D58F3A85BE8582802D47098FB357E5
:103D1800E400B207130755013317E400B183D1B7A4
:103D2800C167637EF5029307F00F1307000263EC87
:103D3800A700972700009387E783AA9703C5070082
:103D48003305A740828021819727000093878782C7
:103D5800AA9703C5070061473305A7408280B707C4
:103D68000001636EF50061819727000093878780C3
:103D7800AA9703C5070021473305A74082804181E0
:103D8800971700009387077FAA9703C50700414745
:103D98003305A7408280B3C7A5008D8B3307C500C4
:103DA80081E78D4763EEC700AA876370E50A83C67B
:103DB800050085078505A38FD7FEE3EAE7FE828025
:103DC80093763500AA8791CA83C6050085078505BD
:103DD800A38FD7FE93F63700FDB79376C7FF1386F8
:103DE80006FE63F0C70683A3050083A2450083AFE0
:103DF800850003AFC50083AE050103AE450103A3EB
:103E0800850183A8C5019385450223A0770003A8EF
:103E1800C5FF23A2570023A4F70123A6E70123A87F
:103E2800D70123AAC70123AC670023AE17019387E4
:103E3800470223AE07FF75B790419107910523AE5E
:103E4800C7FEE3EBD7FEE3E4E7F6828039713EDA9A
:103E58002ED232D436D63AD842DC46DE93878180D9
:103E680022CC804326CA06CEAA8409C41C4C99E3F6
:103E78002285A1250C4454102686228536C6EF00DB
:103E8800902CF2406244D24421618280011126CAFA
:103E98004AC806CE22CC4EC652C4AA842E8901C571
:103EA8001C4D91E3192D9C4C804499E326853125BE
:103EB800971700009387077E631CF402C04083575E
:103EC800C400A18BB1C71C48A1C7FD59294A1C448D
:103ED80083450900FD17B1E91CC463DE0706228685
:103EE800A9452685A122FD576308F502294535A075
:103EF800971700009387077C6314F4008044C1B7C8
:103F08009717000093870777E31BF4FAC04445BF6F
:103F1800A2852685392455D97D55F2406244D2447C
:103F28004249B249224A056182801CC4050963D707
:103F38000700184C63CBE700638945011C401387D1
:103F4800170018C02380B70059B722862685F9289C
:103F5800E31F35F7D1B71C401387170018C029474E
:103F68002380E70061B793878180AA85884339BF9A
:103F7800411122C42E848395E50006C6EF10800106
:103F8800634905007C48AA977CC8B2402244410195
:103F980082808357C4007D777D17F98F2316F4003C
:103FA800EDB783D7C500011122CC26CA4AC84EC630
:103FB80006CE93F70710AA842E843289B68991C752
:103FC8008395E50089460146A5258357C4007D777A
:103FD8007D17F98F2316F4008315E4006244F2403C
:103FE800CE864A86B24942492685D2440561FDA853
:103FF800411122C42E848395E50006C6152DFD5770
:104008000357C400631BF500FD77FD17F98F2316CE
:10401800F400B2402244410182808567D98F23167B
:10402800F40068C8FDB78395E50011A4011122CCFE
:1040380026CA4AC806CE4EC6AA842E89328401C52D
:104048001C4D91E39D29971700009387A764631976
:10405800F406C0401C4C1CC48357C400A18BC9C3C0
:104068001C48BDCF1C4808409379F90F1379F90F04
:104078001D8D5C486346F500A285268505262DE53D
:104088001C440505FD171CC41C401387170018C0E5
:10409800238037015C486389A7008357C400858B58
:1040A80081CBA9476316F900A2852685C52C0DED9D
:1040B800F24062444A85D2444249B249056182804D
:1040C800971700009387075F6314F400804459B77B
:1040D800971700009387075AE31EF4F6C0449DBF64
:1040E800A28526853D283DDD7D59D9B7411122C4D9
:1040F8002A842E85B285368697F7FF1F23AA07F0F4
:1041080006C6EFE0DFF6FD576319F50097F7FF1FC6
:10411800938707F09C4391C31CC0B24022444101DD
:10412800828041119387818026C2844322C44AC079
:1041380006C62A892E8489C49C4C99E32685B52E07
:104148009717000093870755631CF402C0400317B4
:10415800C40093170701C18393F68700B5EE93F661
:1041680007019DEEA5472320F900136707042316CE
:10417800E4007D55B24022449244024941018280C4
:1041880097170000938707536314F4008044C1B75E
:10419800971700009387074EE31BF4FAC04445BF06
:1041A800918B8DC74C5889C9930744046384F500E3
:1041B8004A857523232A04028357C4002322040056
:1041C80093F7B7FD2316F4001C481CC08357C4009E
:1041D80093E787002316F4001C4881EF8357C40037
:1041E8001307002093F707286385E700A2854A850F
:1041F800C1298357C40013F7170005C75C48232457
:104208000400B307F0401CCC1C480145A5F78317F0
:10421800C40013F7070839DF93E707042316F400EF
:1042280089BF898B014791E3584818C4F1BF4111F0
:1042380022C42A842E8597F7FF1F23AB07DC06C606
:10424800EF009063FD576319F50097F7FF1F9387F9
:1042580027DC9C4391C31CC0B240224441018280A8
:1042680083D7C500011122CC26CA06CE4AC84EC63D
:1042780013F78700AA842E8471EFD841634DE000BC
:10428800B841634AE0000145F2406244D2444249E1
:10429800B2490561828058547DD703A904009396DA
:1042A800370123A0040063DD060670488357C40065
:1042B800918B99C75C401D8E5C5899C33C401D8EFC
:1042C8005C540C50814626858297FD570357C400DD
:1042D800631DF5009440F54763E8D706B70740200B
:1042E8008507B3D7D700858BA5C31C4823220400B4
:1042F8001CC09317370163D80700FD576314F500F6
:104308009C4091E368C84C5823A02401ADDD930775
:1043180044046384F50026859921232A0402A5B75D
:104328000C500146854626850297FD572A86E31FCD
:10433800F5F69C40A5DF75476385E7005947639408
:10434800E70423A0240181B7136707042316E400B8
:104358007D551DBF83A90501E38709F203A905005F
:104368008D8B23A0350133093941014791E3D849A1
:1043780018C4E35A20F11C540C50CA864E86268570
:1043880082976349A0008357C40093E70704231664
:10439800F4007DBFAA993309A940E1BF9C49B9CF70
:1043A800011122CC06CE2A8411C51C4D81E72EC6E8
:1043B8002922B245971700009387C72D639BF50004
:1043C8004C408397C50095C722856244F240056139
:1043D80041BD971700009387E72D6394F5000C44BF
:1043E800CDB7971700009387E728E39CF5FC4C446A
:1043F800C9BFF2406244014505618280014582805F
:10440800411122C406C62A842316B5002317C50005
:104418002320050023220500232405002322050666
:1044280023280500232A0500232C05002146814561
:104438001305C505EFC0BFA497070000938787B38E
:104448005CD097070000938707B61CD49707000035
:10445800938747BA5CD497070000938707BD00D0BD
:104468001CD8B24022444101828097050000938500
:1044780025F389AA411126C2130680069384F5FF05
:10448800B384C4024AC02E8922C406C69385440751
:104498009D2E2A8401CD23200500232225013105E4
:1044A80008C4138684068145EFC07F9D2285B240EB
:1044B800224492440249410182801C4DBDE34111CE
:1044C80006C622C497070000938767FA1CD597177A
:1044D80000009387E7249C4323240504232605042E
:1044E800232805046314F50085471CCD2A841D285C
:1044F80048C02285052808C422852D2048C4484084
:1045080001469145F53D08440546A545D53D484435
:104518000946C945F53585471CCCB24022444101BE
:10452800828082804111971700009387671F26C2F7
:1045380084434AC006C69C4C22C42A8999E326852E
:10454800AD3F938484048044DC40FD1763D60700A4
:104558009C40B9CF8440C5BF0317C40039E7C17771
:104568008507232204062320040023220400232491
:1045780004005CC423280400232A0400232C04001C
:10458800214681451305C405EFC07F8F232A040205
:10459800232C040223240404232604042285B24085
:1045A800224492440249410182801304840671BF67
:1045B80091454A85C13588C051FDB1472320F9008E
:1045C8000144E9BF797122D44AD052CC56CA5AC89C
:1045D8005EC606D626D24ECE2A8AAE8A1304850433
:1045E8000149054BFD5B09ECB25022544A859254AF
:1045F8000259F249624AD24A424BB24B4561828023
:10460800044483294400FD1963D409000040E1BF34
:1046180083D7C400637BFB008397E400638777013B
:10462800A6855285829A3369A90093848406E1BFDE
:10463800411122C42A842E85B285368697F7FF1F3A
:1046480023A8079C06C6EF003026FD576319F5001E
:1046580097F7FF1F9387C79B9C4391C31CC0B24029
:104668002244410182801971A6DAAE848395E5005F
:10467800A2DC86DE328463DC050083D7C40023A075
:10468800060093F7070885E7930700401DA0300848
:1046980036C6EF007016B246E34105FE7247BD67A5
:1046A800F98F7977BA9793B717009CC2F1BF930730
:1046B80000041CC0F6506654D65401450961828036
:1046C80083D7C500011122CC06CE26CA4AC8898BD9
:1046D8002E8489CF930774041CC01CC885475CC806
:1046E800F2406244D244424905618280740030003D
:1046F800AA84953FA2452A892685312201ED831790
:10470800C40013F7072069FFF19B93E727002316DE
:10471800F400C9B797070000938767D59CD48357DF
:10472800C40008C008C893E707082316F400A24786
:104738005CC8B24791CF8315E4002685EF00F00EE0
:1047480001C98357C400F19B93E717002316F400AF
:104758008357C4003369F9002316240151B7DDC11A
:1047680083A7C5FF411122C406C626C21384C5FF0C
:1047780063D307003E94AA84EF00D00F9387C183C8
:104788009C4381EF2322040023AE81822244B2405D
:104798002685924441016F00100E637EF400144098
:1047A8003307D4006396E7009843DC43369718C074
:1047B8005CC0D9BFBA87D84319C3E37DE4FE9443EC
:1047C8003386D700631F86001040B29694C33386A1
:1047D800D700E31DC7FA10435843B29694C3D8C311
:1047E80075B76375C400B1479CC04DB71040B30698
:1047F800C4006316D70014435843B29614C058C077
:10480800C0C369B78280011126CA93843500F19824
:1048180006CE22CC4AC84EC6A104B14763F3F404BD
:10482800B14463E2B4042A89EF00D0049387C183BA
:1048380098433A8439E0938701849C4391E7814502
:104848004A85592723A0A184A6854A85B52FFD59F5
:1048580063193507B1472320F9004A85EF00B001F5
:1048680029A0E3D004FCB1471CC10145F2406244D1
:10487800D2444249B249056182801C40858F63CF8A
:104888000702AD4663F6F6001CC03E9404C031A092
:104898005C406313870223AEF1824A85EF00A07D56
:1048A8001305B4009307440061993307F5405DDFB1
:1048B8003A94898F1CC05DBF5CC3C5B7228740404E
:1048C80095BF130435007198E30285FCB305A44035
:1048D8004A85DD2DE31C35FBB5BF1C46FD171CC6FC
:1048E80063DA0700184E63C5E700A9476394F5002B
:1048F8006FF0CFF31C422E851387170018C2238050
:10490800B7008280011122CC26CA4AC84EC652C4BA
:1049180006CE2A89AE893284B304D6007D5A631440
:104928009400014509A8834504004E864A857537D9
:104938000504E31645FFF2406244D2444249B249B5
:10494800224A05618280357122CD26CB4AC94EC7DD
:1049580006CF52C556C35AC1DEDEE2DCE6DAAA89C2
:10496800AE843289368409C51C4D99E3EFF0FFB453
:1049780097170000938707D2639BF40C83A4490020
:1049880083D7C400A18BF5C79C48E5C793070002ED
:10499800A304F1029307000302D22305F10222C601
:1049A800930B5002971A0000938ACAD2054C294BE0
:1049B8004A848347040099C36390770FB30C24415A
:1049C800638D0C00E6864A86A6854E85253FFD57F1
:1049D8006306F51E9256E69636D283470400638F27
:1049E800071CFD571309140002C802CE3ECA02CCA8
:1049F800A309010482D48345090015465685B12DC3
:104A080013041900C24759E913F7070109C7130727
:104A18000002A309E10413F7870009C71307B002CE
:104A2800A309E104834609001307A0026380E6088E
:104A3800F2474A848146254603470400930514003B
:104A4800130707FD6379E60AB5CA3ECE85A897170E
:104A58000000938727C66395F40083A489000DB7E7
:104A680097170000938707C1E39CF4F083A4C9005B
:104A780001BFA6854E85EFF0CFEA09D97D55FA40EA
:104A88006A44DA444A49BA492A4A9A4A0A4BF65BBE
:104A9800665CD65C0D618280050421BF33055541F3
:104AA8003315AC00C98F3EC82289B1B73247930687
:104AB8004700184336C6634907023ACE0347040045
:104AC8009307E002631FF704034714009307A0024B
:104AD800631BF702B2470904138747009C433AC691
:104AE80063C107023ECA35A83307E04093E72700B1
:104AF8003ACE3EC8E1B7B387670385462E84BA9796
:104B080025BFFD57C5B7050402CA8146814725461A
:104B18000347040093051400130707FD6376E606B0
:104B2800F1F2834504000D4617150000130505BB77
:104B38002D2311CD97170000938747BA1D8D930732
:104B48000004B397A700424505045D8D2AC8834534
:104B58000400194617150000130585B81309140039
:104B68002304B102DD293DC197B7FFFF93870749A9
:104B780095E74247B2471377071009CF91073EC61A
:104B88009257D2973ED22DB5B387670385462E84B8
:104B9800BA97BDBF9D07E19BA107D5B778009706D7
:104BA8000000938666D626860C084E85970000007E
:104BB800E7000000FD572A8AE314F5FC83D7C400F8
:104BC80093F70704E39C07EA125555BD780097064A
:104BD8000000938666D326860C084E85012AD9BF25
:104BE800797156CA9C49BA8A984522D426D24ECEA3
:104BF80052CC06D64AD05AC85EC6AA892E84B28438
:104C0800368A63D3E700BA879CC00347340419C3C4
:104C180085079CC01C4093F7070281C79C40890701
:104C28009CC00329040013796900631A0900130B57
:104C38009401FD5B5C449840998F634CF9041C40D7
:104C48008346340493F70702B336D000A5EB130666
:104C58003404D2854E85829AFD576303F5041C40BF
:104C680011469840998B544481446397C700B38494
:104C7800E64063D3040081441C4418486354F70099
:104C8800998FBE94014969047D5B639824050145A9
:104C980009A885465A86D2854E85829A631E750173
:104CA8007D55B250225492540259F249624AD24A6E
:104CB800424BB24B456182800509ADBF3307D40032
:104CC80013060003A301C70403475404938716007F
:104CD800A2978906A381E7049DBF85462286D285CF
:104CE8004E85829AE30E65FB050945B7797122D492
:104CF80026D24AD04ECE06D652CC56CA5AC8B68903
:104D080083C68501930790063289AA842E84138668
:104D18003504638DF60263E2D7069307800563873F
:104D2800F61863EDD7006380062293073004638E7C
:104D3800F60A930A24042301D404C9A09307300671
:104D48006385F60A93074006E395F6FE1C40084380
:104D580093F6070893054500C5C61C410CC363D8E4
:104D680007001307D002B307F040A301E404971625
:104D780000009386669729476DA893070007638309
:104D8800F61663E5D7029307E006638AF6189307D9
:104D9800F006E390F6FA0C401C4313F80508138557
:104DA80047006307080608C39C438DA8930750076C
:104DB800E383F6FE93078007638AF61293073007AA
:104DC800E399F6F61C43D04181459386470014C306
:104DD80083AA07005685512401C53305554148C0AB
:104DE8005C401CC8A301040471A81C43930A240452
:104DF800938647009C4314C32301F4048547D5B721
:104E080093F607041C410CC3B9DAC207C18781BFF6
:104E180093F5050408C3C9D983D707001307F0061B
:104E28006387E60E971600009386068C2947A30130
:104E380004044C400CC463C5050008406D9908C0C3
:104E480099E3B28A91CDB28AB3F5E702FD1AB69515
:104E580083C505002380BA00B3D5E70263FFE70ADC
:104E6800A147631EF7001C40858B91CB58401C4816
:104E780063C7E70093070003A38FFAFEFD1A330602
:104E8800564110C84E87CA867000A2852685893B80
:104E98007D5A631E450B7D55B250225492540259D7
:104EA800F249624AD24A424B45618280A382D504C4
:104EB80097160000938646830C40084313F80508AC
:104EC8001C411105630D080208C313F7150001C73B
:104ED80093E505020CC04147B9FB0C4093F5F5FD7D
:104EE8000CC0B1B79C4193E707029CC193078007A8
:104EF800A302F404971600009386468075BF13F842
:104F0800050408C3E30308FCC207C1837DBF9706F5
:104F180000009386667D214719BFAE8735B7944157
:104F28001C43CC4913F8060813854700630608009C
:104F380008C39C438CC301A808C393F606049C438A
:104F4800F5DA2390B70023280400B28A25BF144855
:104F58005686CA8526858299E30F45F31C40898BBE
:104F68008DE7B2474844E359F5F23E8535B78546A3
:104F78005686CA8526858299E30F65F1050A5C4441
:104F88003247998FE345FAFEE9BF014A930A940133
:104F98007D5BF5B7411122C42A842E85B2853686F9
:104FA80097E7FF1F23A6070606C63922FD57631990
:104FB800F50097E7FF1F9387A7059C4391C31CC083
:104FC800B240224441018280411122C42A842E85A4
:104FD80097E7FF1F23AE070206C6FD20FD5763199A
:104FE800F50097E7FF1F9387A7029C4391C31CC056
:104FF800B240224441018280411122C42A842E8574
:10500800B28597E7FF1F23A5070006C6B528FD57F9
:105018006319F50097E7FF1F938787FF9C4391C3A8
:105028001CC0B240224441018280411122C42A841A
:105038002E8597E7FF1F23AD07FC06C6B128FD574D
:105048006319F50097E7FF1F938787FC9C4391C37B
:105058001CC0B24022444101828093F5F50F2A9684
:105068006314C5000145828083470500E38DB7FEC0
:105078000505FDB7828082809307800517E7FF1F2B
:105088002328F7F87D5582809307800517E7FF1FCF
:105098002320F7F87D5582809307800517E7FF1FC7
:1050A8002328F7F6014582809307800517E7FF1F3D
:1050B8002320F7F67D5582809307800517E7FF1FA9
:1050C8002328F7F47D558280938741849C4391C7B8
:1050D8003E9523A2A1843E85828097E7FF1F938790
:1050E80067F33E9523A2A1843E8582803C3E3E3EE6
:1050F8003E3E3E3E3E4F6E5278446F6E650A0D004E
:105108005258453C3E3E3E3E3E3E3E3E0A0D000065
:105118003C3E3E3E3E3E3E3E3E4F6E527854696DAA
:10512800656F75740A0D00003C3E3E3E3E3E3E3EB5
:105138003E4F6E5478446F6E650D00003C3E3E3E17
:105148003E3E3E3E3E5458450A0D00002E2E2E503F
:10515800696E67310D0000003132333435000000CC
:1051680055415254200D000066616C673D25640D61
:105178000A0000006C696E65206565720D0000000C
:10518800545249470D00000054696D65206F7574CD
:105198000D00000062756666727420656D70747922
:1051A800200D00002B2B2B4750494F425F4952518D
:1051B80048616E646C65722B2B2B200D000000007B
:1051C8005254432054696D696E672E2E2E200D00AF
:1051D800C4170000E0120000FA170000D013000006
:1051E80060140000141500009E150000B41500009E
:1051F8007A1600009016000002170000D012000076
:10520800D4170000DE1E00005E180000FE18000023
:10521800B61900004E1A0000201900009A19000063
:1052280060190000361E0000C21F0000482400005C
:10523800881F000034240000D223000090240000BE
:10524800A6260000CE17000018180000201800003D
:1052580080180000EC2300009A180000D018000005
:10526800EA180000F4180000181900007E19000060
:10527800361B0000BA1B00000A1E00007C1E00003E
:105288009C1E0000BE1E0000F61E0000021F00004B
:105298002C1F0000461F0000621F00007E1F000038
:1052A800402000006C2000009E200000EA20000042
:1052B800F4200000262100004A210000842100007B
:1052C800BE210000E82100002E2200007622000006
:1052D800BA220000EA24000046230000FE22000053
:1052E80080230000B8230000EE25000064130000AE
:1052F8007761697420627573792070696E207469AA
:105308006D656F75740D0000D6C6FFFFEAC6FFFF16
:10531800EAC6FFFF14C7FFFF24C7FFFF00C7FFFF50
:1053280000C7FFFF00C7FFFF00C7FFFF00C7FFFF61
:1053380000C7FFFF00C7FFFF00C7FFFF00C7FFFF51
:1053480000C7FFFF34C7FFFF2EC7FFFF6EC7FFFF71
:105358006EC7FFFF9AC7FFFFC4C7FFFF5AC7FFFF0B
:105368005AC7FFFF5AC7FFFF5AC7FFFF5AC7FFFFB9
:105378005AC7FFFF5AC7FFFF5AC7FFFF5AC7FFFFA9
:105388005AC7FFFFE2C7FFFF5CC8FFFF0EC9FFFF58
:105398000EC9FFFF42C9FFFFE2C9FFFF06C9FFFFB1
:1053A80006C9FFFF06C9FFFF06C9FFFF06C9FFFFC1
:1053B80006C9FFFF06C9FFFF06C9FFFF06C9FFFFB1
:1053C80006C9FFFF68CAFFFF4AD3FFFF0ED4FFFFDD
:1053D80068D5FFFF4AD3FFFF4AD3FFFF0000000054
:1053E800CDCCCCCCCCCCF83F0000000000009940DC
:1053F8000000000000408F4000000000A3E1E140F1
:105408000000000000003440000000000000594087
:105418007061796C6F61644C656E6774683D256C6A
:10542800640D0A004D4F4445205F2052580D00007E
:10543800697271526567733D25640D0A00000000AA
:105448004D4F4445205F2052585F444F4E450D0054
:105458002B2B2B2B2B2B2B2B2B2B4D4F4445202031
:1054680054582B2B2B2B2B2B2B2B2B2B2B200D0082
:1054780036363636363636363636363636363636C4
:105488003636363636363636363636363636360DDD
:105498000000000036373737373737373737373771
:1054A800373737373737373737370D006E6F206361
:1054B8006F6D6520696E202073776963680D000041
:1054C80000000000A8CB684054D8FFFF7CD8FFFF3D
:1054D800A4D8FFFFBCD8FFFFD6D8FFFFE6D8FFFF50
:1054E8000ED9FFFF36D9FFFF4ED9FFFF68D9FFFF5E
:1054F800E0DEFFFF64DDFFFF74DEFFFF7CDEFFFF01
:1055080074DEFFFF94DDFFFF74DEFFFF7CDEFFFF2C
:1055180064DDFFFF64DDFFFF94DDFFFF7CDEFFFF3E
:10552800D6DEFFFFD6DEFFFFD6DEFFFF94DDFFFFEE
:105538001AE4FFFF10E3FFFF10E3FFFF0EE3FFFF96
:1055480016E3FFFF16E3FFFFDCE2FFFF0EE3FFFFBA
:1055580016E3FFFFDCE2FFFF16E3FFFF0EE3FFFFAA
:1055680006E4FFFF06E4FFFF06E4FFFFDCE2FFFFBF
:1055780000010202030303030404040404040404F2
:1055880005050505050505050505050505050505C3
:1055980006060606060606060606060606060606A3
:1055A8000606060606060606060606060606060693
:1055B8000707070707070707070707070707070773
:1055C8000707070707070707070707070707070763
:1055D8000707070707070707070707070707070753
:1055E8000707070707070707070707070707070743
:1055F8000808080808080808080808080808080823
:105608000808080808080808080808080808080812
:105618000808080808080808080808080808080802
:1056280008080808080808080808080808080808F2
:1056380008080808080808080808080808080808E2
:1056480008080808080808080808080808080808D2
:1056580008080808080808080808080808080808C2
:1056680008080808080808080808080808080808B2
:105678000000000000000000000000000000000022
:105688000000000000000000000000000000000012
:105698000000000000000000000000000000000002
:1056A80000000000000000000000000000000000F2
:1056B80000000000000000000000000000000000E2
:1056C80000000000000000000000000000000000D2
:1056D800232D302B20000000686C4C006566674560
:1056E8004647000030313233343536373839414295
:1056F80043444546000000003031323334353637F4
:10570800383961626364656600000000CE09D30918
:10571800D8090000CF09D409D9090000F80D0020E4
:10572800A41100002E0F000000000000000000007F
:10573800C4110000E4110000440F00000000000044
:10574800000000000000000098560000B856000055
:105758007856000000000000000000000000000073
:105768000000000000000000000000000000000031
:105778000000000000000000000000000000000021
:105788000000000000000000000000000000000011
:105798000000000000000000000000000000000001
:1057A80000000000140041400C2A0000F80D002001
:0857B80000000000AABBCCDDDB
:00000001FF
